:020000040000FA
:1000000000004F3094001E28831A0D281710950009
:10001000030E960004089800942883121714950084
:10002000030E960004089800942818088400160E01
:100030008300950E150E17188316090014308400DE
:100040003B309100840A8001910B222864280530FE
:10005000030503190800053C080010080E02031DE3
:1000600008000F088D0208003C200F088D070318B8
:100070008E0A10088E0708008F0990093F288F0FFD
:100080000800900A08008F00472891178E1F9113CF
:100090005320031908000310911B03148E0C8D0CC0
:1000A0008F0B4B2808000F0810040800840000087C
:1000B0008D00840A00088E000800840000088F006C
:1000C000840A0008900008004E30A6008A018301CF
:1000D000692883167F308105C73081050830810487
:1000E00083128101A501FF308604FB308B05831646
:1000F000F33086058312F7308605FB30860598209D
:1001000080308B04251C8728FE30A505A2210B1DFD
:100110008D28FB308B05C921B521A51C9228FD3007
:10012000A505A3219E208228962815289528080039
:100130000130A90004309F00A00108000530290209
:10014000031DB3280608FF3A8D008D1CB3281D300F
:10015000562009308F0090012D2027200319B32845
:10016000BF219D019E0101302902031DFC281D3085
:10017000562020308F004E3090002D200318ED289F
:100180000608043886001E1ED92804309F00A001EE
:1001900023305D201D30562034201F305D202D205F
:1001A00027200319D828BF211D08A3001E08A4007A
:1001B000EC2802309F00A00123305D201D30562026
:1001C00034201F305D202D2027200319EC28BF216B
:1001D0001D08A3001E08A400F0280608FB398600AD
:1001E0001D30562040308F009C3090002D2027205D
:1001F0000319FC289D019E0102302902031D452997
:100200001D30562020308F004E3090002D200318D6
:1002100036290608043886001E1D222903309F0057
:10022000A00123305D201D30562034201F305D207A
:100230002D20272003192129BF211D08A3001E08F6
:10024000A400352901309F00A00123305D201D301E
:10025000562034201F305D202D20272003193529FA
:10026000BF211D08A3001E08A40039290608FB3978
:1002700086001D30562040308F009C3090002D208D
:100280002720031945299D019E0103302902031DE2
:1002900087291D30562020308F004E3090002D20B1
:1002A000031878290608043886001D3056200330CC
:1002B0008E050D08A1000E08A2002130562008303E
:1002C0008F00900147200D08A1000E08A2002330E6
:1002D0005D201D305620342021305D202D20272028
:1002E00003197729BF211D08A3001E08A4007B293C
:1002F0000608FB3986001D30562040308F009C30A8
:1003000090002D202720031987299D019E0104308C
:100310002902031DA12906080438860002309F0027
:10032000A00123305D201D30562034201F305D2079
:100330002D2027200319A129BF211D08A3001E0875
:10034000A400080008000608FB3986009D019E01F4
:10035000A301A4012908013EA90005302902272094
:100360000319B4290130A90008001D3056208E0A57
:100370008D0F8E030D089D000E089E000800861D3F
:10038000C5290608F7398600C829060808388600F6
:100390000800A60BCF294E30A600D021EA21080084
:1003A000A708031DD72906180800B230E729A71BA4
:1003B000DB29A7030800061CE0290330A70008007A
:1003C00027037F39A700A717031D0800B230A70035
:1003D000A5140800A808031DF12986180800B230EA
:1003E000012AA81BF529A8030800861CFA29033056
:1003F000A800080028037F39A800A817031D0800DB
:08040000B230A8002514080029
:00000001FF
